:020000020000FC
:1000000067C013C013C043C043C043C043C043C014
:1000100043C043C043C052C052C052C052C052C07D
:1000200052C052C052C052C052C018951FB71F9341
:100030000F93713001F1C59A71E0B49B1FC0839595
:10004000843611F480E0C69A891709F4C69806B37D
:1000500003700A1771F0A33061F4B09904C09136AF
:1000600011F00AF49395B19921F4933011F00AF04C
:100070009A95A02F08C0C59870E005C0B39B02C038
:10008000C69A01C0C6980F911F911FBF1895189569
:100090001895189518951895189518950A95002390
:1000A00039F41A95112321F401E0C79809BF05C05E
:1000B000B79B02C0C79801C0C79A189518951895A4
:1000C00018951895189518951895189518951895C8
:1000D00008E00EBF0FE50DBF0FEF0ABB0CEC0BBB2A
:1000E0000FE108BB00EE07BB0FE108BB0FEF04BB3D
:1000F0000CEC05BB00E001BB00E002BB21E031E0FD
:1001000041E051E001E009BF0AEF02BF02E003BF96
:1001100092E3789405D2B29BFECF60FD04C0819B30
:100120007CC061607AC0819978C06E7F809B3BC043
:100130002395283009F420E0203081F1213049F165
:10014000223011F12330D9F02430A1F0253069F0AC
:10015000263031F027300BB3007F01600BBB5DC050
:100160000BB3007F03600BBB58C00BB3007F026072
:100170000BBB53C00BB3007F06600BBB4EC00BB371
:10018000007F04600BBB49C00BB3007F0C600BBB4E
:1001900044C00BB3007F08600BBB3FC00BB3007FB4
:1001A00009600BBB3AC0203009F428E02A952030C2
:1001B00091F02130A9F02230C1F02330D9F0243061
:1001C000F1F0253009F1263021F127300BB3007F03
:1001D00001600BBB22C00BB3007F09600BBB1DC0CD
:1001E0000BB3007F08600BBB18C00BB3007F0C6023
:1001F0000BBB13C00BB3007F04600BBB0EC00BB373
:10020000007F06600BBB09C00BB3007F02600BBB15
:1002100004C00BB3007F03600BBB61FD04C0839B74
:100220007CC062607AC0839978C06D7F829B3BC03E
:100230003395383009F430E0303081F1313049F114
:10024000323011F13330D9F03430A1F0353069F06B
:10025000363031F037300BB30F7000610BBB5DC02F
:100260000BB30F7000630BBB58C00BB30F70006271
:100270000BBB53C00BB30F7000660BBB4EC00BB370
:100280000F7000640BBB49C00BB30F70006C0BBB4D
:1002900044C00BB30F7000680BBB3FC00BB30F70B3
:1002A00000690BBB3AC0303009F438E03A95303081
:1002B00091F03130A9F03230C1F03330D9F0343020
:1002C000F1F0353009F1363021F137300BB30F70D2
:1002D00000610BBB22C00BB30F7000690BBB1DC0CC
:1002E0000BB30F7000680BBB18C00BB30F70006C22
:1002F0000BBB13C00BB30F7000640BBB0EC00BB372
:100300000F7000660BBB09C00BB30F7000620BBB14
:1003100004C00BB30F7000630BBB62FD04C0859B70
:100320007CC064607AC0859978C06B7F849B3BC039
:100330004395483009F440E0403081F1413049F1C3
:10034000423011F14330D9F04430A1F0453069F02A
:10035000463031F0473005B30F70006105BB5DC01A
:1003600005B30F70006305BB58C005B30F70006282
:1003700005BB53C005B30F70006605BB4EC005B387
:100380000F70006405BB49C005B30F70006C05BB5E
:1003900044C005B30F70006805BB3FC005B30F70C4
:1003A000006905BB3AC0403009F448E04A95403046
:1003B00091F04130A9F04230C1F04330D9F04430DF
:1003C000F1F0453009F1463021F1473005B30F70A7
:1003D000006105BB22C005B30F70006905BB1DC0DD
:1003E00005B30F70006805BB18C005B30F70006C33
:1003F00005BB13C005B30F70006405BB0EC005B389
:100400000F70006605BB09C005B30F70006205BB25
:1004100004C005B30F70006305BB63FD04C0879B78
:100420007CC068607AC0879978C0677F869B3BC034
:100430005395583009F450E0503081F1513049F172
:10044000523011F15330D9F05430A1F0553069F0E9
:10045000563031F0573005B3007F016005BB5DC0F9
:1004600005B3007F036005BB58C005B3007F026081
:1004700005BB53C005B3007F066005BB4EC005B386
:10048000007F046005BB49C005B3007F0C6005BB5D
:1004900044C005B3007F086005BB3FC005B3007FC3
:1004A000096005BB3AC0503009F458E05A95503005
:1004B00091F05130A9F05230C1F05330D9F054309E
:1004C000F1F0553009F1563021F1573005B3007F76
:1004D000016005BB22C005B3007F096005BB1DC0DC
:1004E00005B3007F086005BB18C005B3007F0C6032
:1004F00005BB13C005B3007F046005BB0EC005B388
:10050000007F066005BB09C005B3007F026005BB24
:1005100004C005B3007F036005BBFDCDFFCFFFCF57
:1005200002E005BD00E409BF1AE00FEF0000000083
:0A0530000000F9B6F6FCFACF0895BA
:00000001FF
